:0300000002128A5F
:03000B000200C12F
:03002B000203CB02
:03005B0002059803
:0300730002058EF5
:1000800002030406080C10182030406080020304AC
:1000900006080C101820304080FF0406080C1018C9
:1000A0002030406080A0C000000001010003020277
:1000B000010D0D040206020D0505050D06030502DE
:1000C00002C2AFC0D0C0E0205A0D302F02E473301E
:1000D000600280F90203B7306306D297D295D293BB
:1000E00085258AC25AE525F4700221AA056130608F
:1000F00013206A19758B00D0E0D0D0D297D295D258
:1001000093D2AF32D297D295D29302019AD26EC2D5
:100110006FE565601CC3E5611495654014C26ED23D
:100120006FC3E5619564500302019A756100020195
:100130009A206C14D297D295D2937401D5E0FDD257
:1001400096D294D29202019AD297D295D293E53D5B
:1001500020E22520E10D207502D296307502D2945E
:1001600002019A20E005D29202019A207502D294EF
:10017000307502D29602019A20E11520E00D20751B
:1001800002D296307502D29402019AD29202019A5A
:10019000207502D294307502D296758B00D0E0D0D3
:1001A000D0D297D295D293D2AF32D0E0D0D0D2AFC6
:1001B0003261B7E525600A207502C297307502C228
:1001C00095D29361B7E5256002C293207502D2955E
:1001D000307502D29761B7E525600A207502C29595
:1001E000307502C297207502D297307502D29561A0
:1001F000B7207502C296307502C294E525600A20C8
:100200007502C297307502C295207502C29430758E
:1002100002C296D29361B7207502C296307502C2AF
:1002200094207502C294307502C2967419D5E0FD0F
:10023000E525600A207502C297307502C295D293F7
:1002400061B7207502C296307502C294E525600A36
:10025000207502C297307502C295C292D29361B7DF
:10026000207502C296307502C294C2927419D5E00C
:10027000FDE525600A207502C297307502C295D24D
:100280009361B7C292E5256002C293207502C296BF
:10029000307502C294207502D295307502D29761F2
:1002A000B7C292207502C296307502C2947419D5F5
:1002B000E0FDE5256002C293207502D295307502FB
:1002C000D29761B7C292E5256002C293207502C23F
:1002D00094307502C296207502D295307502D2977D
:1002E00061B7C292207502C294307502C296741929
:1002F000D5E0FDE5256002C293207502D2953075E8
:1003000002D29761B7207502C294307502C296E599
:1003100025600A207502C295307502C297C29220EC
:100320007502D297307502D29561B7207502C294DA
:10033000307502C296C2927419D5E0FDE525600AB7
:10034000207502C295307502C297207502D297308F
:100350007502D29561B7207502C294307502C296BB
:10036000E525600A207502C295307502C297207596
:1003700002C296307502C294207502D2973075027F
:10038000D29561B7207502C294307502C29620756D
:1003900002C296307502C2947419D5E0FDE525605D
:1003A0000A207502C295307502C297207502D29755
:1003B000307502D29561B7E525F4F58A758B007525
:1003C0006000D25AD0E0D0D0D2AF32C2AFC0D0C0DD
:1003D000E0D2D3C2CEE528600A741F552E604915BD
:1003E00028812878007900E580307601F430E50234
:1003F00078FF53DACF20760343DA2030760343DAEE
:1004000010C2D8C269E580307601F430E50279FF88
:10041000C3E89970CE305903752840741F552E607B
:10042000037528408858D268E52960041529813B66
:10043000741F552E600543DA01C2D820680281C0BE
:10044000E558F8C268741F552E60367982B70431BA
:10045000C3E894F0400374F0F8E8C4540F28F87926
:1004600084B703028181C313C3138721200802C309
:0E04700013200A06C3C898F8818128F85003AB
:10047E0074FFF8C3E8955F5003E55FF8E52C54066A
:10048E007030882230630AC3E522955C4003855C98
:10049E00227882B6041CC3E5229524401278A096D9
:1004AE00400DE52426F52450097524FF0204C0856D
:1004BE00222420CF09D0E0D0D0C2D3D2AF32C2CFC7
:1004CE007801E5286008741F552E70021528C3E5C3
:1004DE005894014005755B0081EFE55B04600205F1
:1004EE005B7982B7020EE548601EC3E52294324066
:1004FE00178547227982B7030FE548600BC3E522C3
:10050E0094324004798E8722C3E5239522600840F9
:10051E00041523A1250523D8C80562E562700215CE
:10052E0062D563537563017803C3E562941E404739
:10053E00C3E562946450087801756303020559C3DC
:10054E00E562949650057801756301C3E55D9524C7
:10055E004018E548701485245DE5620460037562F9
:10056E001E75630175233C020585C3E55D285005A4
:10057E00755DFFA185F55DD0E0D0D0C2D3D2AF328C
:10058E00C2AF53917FC258D2AF32C2AFC0D0C0E01B
:10059E00C0F0D2D3A8FBA9FCC2D8306902A1FB538C
:1005AE00DACF20760343DA1030760343DA20D269AD
:1005BE00E580307601F420E502A1CF88268927E177
:1005CE009B53DACF20760343DA2030760343DA10DA
:1005DE00C2D8C269741F552E7002E1817800E58081
:1005EE00307601F430E502E1818858E18153DACFAB
:1005FE0020760343DA2030760343DA10C26920599D
:10060E0002C1B553DACF20760343DA1030760343B6
:10061E00DA20C2D8D26988538954C3E89551F8E9D3
:10062E009552F9E4FB7AFAC3E894C8E994005008AD
:10063E00E4D2E4FB7A0AC188C3E89468E9940150D5
:10064E0008E4D2E3FB7A0FC188C3E894D0E99402A0
:10065E005008E4D2E2FB7A1EC188C3E894A0E99464
:10066E00055008E4D2E1FB7A3CC188C3E89498E9CE
:10067E0094085006E4D2E0FB7A78C3E89555FCE97D
:10068E009556FD30E708ECF42401FCEDF4FD7557AA
:10069E00007008C3EC9A500375570188558956A807
:1006AE0053A95488518952C3E89526F8E99527F93C
:1006BE00307402E154307302E154307202E14DE9BC
:1006CE00C313F9E813F8307102E14DE9C313F9E8E9
:1006DE0013F8307002E14DE9C313FDE813FC205905
:1006EE0018C3EC941CED94024003020781ED7009CF
:1006FE00C3EC94C8500302079B74002077037896CE
:10070E00E624FAFEE43400FFC3EC9EFCED9FFD50A0
:10071E000678007900E154C3EC94FFED9400400696
:10072E0078FF7900E154EC856CF0A4C5F0A2F733A4
:10073E00F87900400302077078FF7900020770E92C
:10074E00C313F9E813F830740EE9600278FFC3E8BA
:10075E001338F8E43400F9C3E894FFE9940040023A
:10076E0078FF8858D268205902E181741FF4552E03
:10077E004BF52E752840741F552E700375280A30C0
:10078E005902E19B741F552E600353DAFE75292022
:10079E00741F552E700375290AD0F0D0E0D0D0C248
:1007AE00D3D2AF327901E1CA7903E1CA790AE1CA3B
:1007BE00791EE1CA7964E1CA79C8E1CA7817E4D52D
:1007CE00E0FDD8FAD9F6227A147B780207F17A1076
:1007DE007B8C0207F17A0D7BB40207F17A0B7BC892
:1007EE000207F1AC257525017902B275E4C292D5E6
:1007FE00E0FDE5256002C293D5E0FDD293D5E0FD84
:10080E00D292D5E0FDE525600A207502C2973075BB
:10081E0002C295E56DD5E0FD207502D297307502C6
:10082E00D2957496D5E0FDD9C1EAF8D5E0FDD8FB96
:10083E00DBB1C2928C2522C37C007D0075F00005D1
:10084E00F0EA33FAEB33FB50F6EB13FBEA13FAC381
:10085E00E9FFE8FEE89AF8E99BF95004EFF9EEF8A3
:0F086E00B3EC33FCED33FDD5F0DFEDF9ECF82200
:10087D00E889F08A20D2D4F8A9F07B0030F70B7B01
:10088D00FFF42401F8E9F43400F9E88520F0A4AD73
:10089D00F0F8E98520F0A4AFF0FEED2EF974003FDD
:1008AD00FA7C04C3EA13FAE913F9E813F8DCF48BC4
:1008BD00F030F70AE8F42401F8E9F43400F9E88996
:1008CD00F0C2D4F8A9F0227882B60403020960C3FD
:1008DD00E55894014018E54870377805C37994B709
:1008ED0002027812C3E53B9400E53C984020E548B0
:1008FD006009855E5D7562FF756301852224E4F5EF
:10090D003FF540F541F542F543F54802096075485C
:10091D0001C37994E79402601BE523F43333F91393
:10092D00F8E9540104F9E854FEC39440F8E9940041
:10093D00F902095CE523F433333333F913F8E95441
:10094D00070404F9E854F8C39440F8E99400F988D1
:10095D003F894022E548603BC3E53C13F9E53B1375
:10096D00F8C3E53F98F8E54099F9500CC3E8948039
:10097D00E994FF401602099CC3E8947FE994005066
:10098D000302099C787F790002099C788079FF88A1
:10099D0044894522E5486058E5442541F8E545354B
:1009AD0042F9854520E4300701F43543FA30E70973
:1009BD00C3EA94F040150209DEC3EA940F50030216
:1009CD0009DE78FF79FF7A0F0209DE780079007A67
:1009DD00F0C3E524955C5006E524600921F7E54553
:1009ED0020E70D21F7E54530E706884189428A4326
:1009FD0022E5487003020A61789EE6FAC3E54433A6
:100A0D00F8E54533F9117DE930E70BC3E89480E94A
:100A1D0094FF40134138C3E8947FE994005002419C
:100A2D0038787F79004138788079FFE820E715C361
:100A3D00E52398F84009C3E894014003020A5F7862
:100A4D0001020A5FE8F424012523F84003020A5F3E
:100A5D0078FF884622E5487003020AC3789FE6FABC
:100A6D00A842A943117DE930E70CC3E89401E9944C
:100A7D00FF4016020A9AC3E894FFE994005003025E
:100A8D000A9A78FF7900020A9A780179FFE920E73E
:100A9D0015C3E54698F84009C3E894014003020ADE
:100AAD00C17800020AC1E8F424012546F84003028A
:100ABD000AC178FF8824227883E6F520121001758B
:100ACD00E890E5E820ECF0A8BDA9BE121099756874
:100ADD0055756900C3740013FD745513FC74552CC2
:100AED00FC74003DFDECFAEDFBC3E89AE99B401464
:100AFD00E5682455F568E5693400F569EA2CFAEBEB
:100B0D003DFB80E5AE68AF69C3E56913F9E5681390
:100B1D00F8C3E913F9E813F8E56828F566E56939CE
:100B2D00F5677A03C3E913F9E813F8DAF7AA201A7F
:100B3D007009756800756900020B581AEA6008EEB5
:100B4D0028FEEF39FFDAF88E688F692275E890225A
:100B5D007883E6FFE5E820ECF7A8BDA9BE056AC3DA
:100B6D00E56A94084052756A00E97007E56B601BF1
:100B7D00020B8CC3E8956B6010E56B5006600C148E
:100B8D00020B980460F9020B98E56BF56BC3946D3D
:100B9D00F84021755CC0C3E89404F84017755C807B
:100BAD00C3E89404F8400D755C40C3E89404F84024
:100BBD0003755C0075BB0822EFC39401601BC3E88D
:100BCD0094FFE994035012C3E89568E995695009BB
:100BDD00E55C600C155C020BEDE55CF46002055CF8
:100BED00A85CC3E524985002A8248825C3E5259563
:100BFD005D400B855D25E55DF46003855D5CC3E5BA
:100C0D006AB4070375BB102230610278323062027C
:100C1D007850E52C5406601FE879A187F0A4C5F043
:100C2D00A2F733F8C3E8955C4002A85C88228824BB
:100C3D008825306102885E22788FE6FFC3EF940528
:100C4D005018C3EF94045020C3EF94035028C3EF02
:100C5D0094025030C3EF940150387533A075340FA2
:0E0C6D0075353C75360581AD7533C075341292
:100C7B0075354075360681AD75337075341775351E
:100C8B00D075360781AD75334C75341D7535C4750C
:100C9B00360981AD7533287534237535B875360B28
:100CAB0081AD85334F853450753B00753C0822A8C8
:100CBB004FA950020CC5A849A94A759100C3E498E5
:100CCB00F594E499F595759104D25875C820A8CC84
:100CDB00A9CD75C824AA39AB3A8839893AC3E89AA1
:100CEB00F8E99BF9AA3BAB3CC3EB13FDEA13FCC33E
:100CFB00ED13FDEC13FCC3EA9CFAEB9DFBEA28FA1F
:100D0B00EB39FB8A3B8B3C400122753BFF753CFF6B
:100D1B0022305802A11C759100C3E4954BF594E465
:100D2B00954CF595759104D258227892E6FF7E107A
:100D3B00305B027F053063047F037E00A93CA83B38
:100D4B007A04C3E913F9E813F8DAF7C3E89EF8E974
:100D5B009400F94009C3E89402E994005004780226
:100D6B00E4F9E9FBE8FAC3E913FDE813FCC3EF94DC
:100D7B0003602EEF20E00DE82CF8E93DF9ECFAEDDD
:100D8B00FB020D99E828F8E939F97A02E4FBC3EF85
:100D9B009403400D8A4D8B4E8849894A8C4B8D4C60
:100DAB0022884D894E8A498B4A8C4B8D4C22305868
:100DBB0002A1B9759100C3E4953BF594E4953CF51C
:100DCB0095759104D25822753E00752000020DE1F5
:100DDB00753E00752040D2AF053E20580122759D0F
:100DEB0000E53CC313C313F8086030306A06C31325
:100DFB00C313F808C3E8940A4002780A306D08C39D
:100E0B00E8940440027804C3E53C9408400D759DBA
:100E1B0002C3E53C94104003759D03205803D2AFE9
:100E2B00227918206D027908D2AF0000C2AF205A88
:100E3B000A7914206D027907306FE03063027978FC
:100E4B00C3E58B9940D5E59BF45440B52002A1E155
:100E5B00D8C9D2AF22C25B789CE6146007E53E147A
:100E6B007002D25B30630B053820581075380002C6
:100E7B000E87205807158115810217D8227591000E
:100E8B00C3E4954DF594E4954EF595759104D258C0
:100E9B0022AE25305B4F78A3E6FFBF010BD25C750A
:100EAB002500D297D295D293B121305C03752500E2
:100EBB00305802C1B5BF020BD25C752500D297D258
:100ECB0095D29378A2B6010DB121305C0375250044
:100EDB00305802C1D5BF030BD25C752500D297D217
:100EEB0095D293D188305C03752500305802C1F040
:100EFB00305B04C25C8E2522C2AFC292206A030211
:100F0B000F25900305206C12306E0F207502C294D2
:100F1B00307502C2967419D5E0FD207502D2963059
:100F2B007502D294759F13753D02D2AF22C2AF20CA
:100F3B006A03020F5A9002C4306E17C292207502D8
:100F4B00C294307502C2967419D5E0FD020F5D9004
:100F5B0001C5207502D295307502D297305A06E53D
:100F6B00256002C293207503759F10307503759F22
:100F7B0011753D03D2AF22C2AF207502C2963075F8
:100F8B0002C294206A03020FA4900283206C0A30E1
:100F9B006E07C2927419D5E0FD207502D29430759C
:100FAB0002D296207503759F11307503759F1075CE
:100FBB003D04D2AF22C2AF206A03020FE29002427D
:100FCB00306E17207502C296307502C294C29274AD
:100FDB0019D5E0FD020FE59001B3D293305A0EE51F
:100FEB0025600A207502C297307502C295759F1352
:100FFB00753D05D2AF22C2AF207502C29430750287
:10100B00C296206A0302102B9001F1206C12306EF5
:10101B000F207502C296307502C2947419D5E0FD8B
:10102B00D292207503759F10307503759F11753D16
:10103B0006D2AF22C2AF206A03021069900356306A
:10104B006E1F207502C296307502C294207502C2C3
:10105B0094307502C2967419D5E0FD02106C9001A4
:0E106B00D7207502D297307502D295305A0EFA
:10107900E525600A207502C295307502C297207570
:1010890003759F11307503759F10753D01D2AF220D
:101099009001B1D297D295D293C296C294C29222AC
:1010A900C3E54F9535E55095365001227890E6FF16
:1010B900C3EF94055018C3EF9404501BC3EF940376
:1010C900501EC3EF94025021C3EF94015024C3E58D
:1010D9004F943CF8021104C3E54F9428F802110417
:1010E900C3E54F941AF8021104C3E54F9412F802AC
:1010F9001104C3E54F940AF8021104E5509400F96C
:10110900884F89502230580302110E2278807607C1
:1011190078817607788276017894760178837604E7
:101129007886760A788F76037890760178957602B4
:1011390078927603789B760D789376017887760294
:10114900789C7601788876017889760178857600A9
:10115900788C7601788D7600788E76B478967625B7
:10116900789776D078987678789976C8789A760448
:10117900789D7600227893E6FF756409756501C349
:10118900BF02097564057565010211C3C3BF03096F
:101199007564057565020211C3C3BF040975640549
:1011A9007565030211C3C3BF050675640975650733
:1011B900C3BF06067564007565007887E6FFC26CD3
:1011C900C3BF0302D26CC26BC26A7418552D600288
:1011D900D26AC26E6002D26ED26F6002C26FC275ED
:1011E9007888E630E102D275C2767889E630E10284
:1011F900D276C3EF94026008758E01D26D02120E89
:10120900758E00C26D227880E61490008093789ED6
:10121900F67881E61490008093789FF611992278E8
:101229009BE61490008D9378A0F61199227886E6B2
:101239001490009A9378A1F6119922789CE614905B
:1012490000A79378A2F6789CE6149000AC9378A353
:10125900F6119922227896E6FA7897E6FB30770418
:101269007A007BFFC3EB9AFCC3948250027C82759F
:101279006C00056CEC856CF0A4C3E5F0948040F239
:1012890022C2D353D9BF7581C043FF801207B275FB
:10129900EF0243B203E5B324044002F5B37580FFBE
:1012A90075A40075F1B275D4DF7590A975A5FC75A3
:1012B900F2FE75D50175A60175E2411199E4F8F6BA
:1012C900D8FD3115121822317E510F51285136514E
:1012D90044515D515E7898866D119975885075896C
:1012E9000275C82475910475D8401207C61207D52E
:1012F9001207BE1207DC1207BE1207E31207BE125D
:101309001CE51207C61207C61207C275A82275B8CE
:101319000275E69075F610759B80759D0375D10E63
:1013290075BC5875BB0875BA1175E8801207B2D239
:10133900AF120AC443DA01C2D8C2691207C67530AE
:1013490001D2597A05E55770027A051207B6E558B0
:10135900C3940240EEE52E541F855A59F55AB559E2
:10136900E2DAE2C25953DACF20760343DA20307643
:101379000343DA10C2D8C2691207C21207B678024B
:10138900741F552E70027800C3E5589840EDC2AF1E
:101399001207D51207D51207D5D2AF1207C675475E
:1013A900001207B6788CE6C394015003021473E562
:1013B90030C394015003021473741F552E6035C352
:1013C900E55894FF5003021473C2AF1207EAD2AF73
:1013D9001207C2C3E558940150EFC2AF1207D512E4
:1013E90007BA1207D5D2AF1207C2C3E55894FF4016
:1013F900E9021D6A7F05D277515E1207C2C2AFC2E8
:1014090077515EC3E558947FD2AF4068C2AF1207E7
:10141900EAD2AFDFE1C3E55894057897F61207C61B
:101429001218D2121CED7F0AD277515E1207C2C27E
:10143900AFC277515EC3E558947FD2AF50E8C2AFCF
:101449001207D51207BA1207D5D2AFDFDBE5582448
:10145900057896F61207C61218D2121D1C1207C279
:0F146900C3E55894FF40F6021D6AC3E558954746
:1014780040038558471207C2C3E5589401400261EA
:10148800AAC2AF1207EA1207EA1207EAD2AF120796
:10149800C6753000E4F531F5320531E531F47036C2
:1014A8000532789AE67828146012785014600D781E
:1014B800A014600878F0146003753200C3E5329810
:1014C800401415327899866DC2AF1207EAD2AF7808
:1014D80098866D1207C21207B6E5287008741F5562
:1014E8002E7002614AC3E558940640AD1207C2E562
:1014F80028700302134A1199E4F522F523F524F51F
:1015080025755CFF7885865FF53FF540F541F54226
:10151800F543F56AF548F52BF52CF55B120C457586
:101528006A0875BB101207B2120B59E5E820ECFBEC
:10153800A8BDA9BEE97001F8886B120B5D756A0831
:1015480075BB107895E630E00302158E7887E6FEC5
:101558007602317E7887EEF6D261C2AF120C15851D
:10156800225C85225DD2AFC2617525007562007567
:101578006301D260D2637538001101113F120CC1AA
:10158800120C450216B07887E6FE76037893E6FDDE
:101598007605317E7887EEF67893EDF6D260D261E3
:1015A800D26E1101113F120C151207B2120F03125D
:1015B80007B21207B2120F381207B6120F821207BB
:1015C800B61207B6120FC01207BA11011207B612E7
:1015D80007B2C261D262120B59120B5D120C15755B
:1015E8006A0875BB10113F120CBA120D3511A931DA
:1015F8000E120F03120CBA120D3511A9310E120F6B
:1016080038120CBA120D3511A9310E120F82120CB4
:10161800BA120D3511A9310E120FC0120CBA120DE3
:101628003511A9310E1101120CBA120D3511A9C3C9
:10163800E54F9535E5509536400C310EC3E5589485
:101648000150930217D8310EC2627887E6FE7602FF
:10165800317E7887EEF685225C855E5D855E257530
:101668006200756301D263753800C2AF207502C28B
:1016780096307502C294207502C294307502C296E3
:10168800742DD5E0FDD2AF113F120CC1120D1C1202
:101698000D35120DB9756A0075BB080216B0317E9A
:1016A800113F756A0075BB08120DDB120E60120E31
:1016B800881208D4120E9C120F03120CC1120D1CB2
:1016C800120D35120DB9120DD2120E60120E8812BB
:1016D8000961120E9C120F38120CC1120D1C120D4A
:1016E80035120DB9120DDB120E60120E881209A107
:1016F800120E9C120F82120CC1120D1C120D351203
:101708000DB9120DD2120E60120E881209FE120EB9
:101718009C120FC0120CC1120D1C120D35120DB9FE
:10172800120DDB120E60120E88120A62120E9C1144
:1017380001120CC1120D1C120D35120DB9120DD269
:10174800120B59120E60120E88120B5D120E9C11AC
:101758003F120CC1120D1C120D35120DB930632A3F
:10176800855E5C855E5D756200756301C3E53894CE
:1017780064400AC263D264753714021792C3E558ED
:10178800940140030216B00217D8306419E53714E3
:101798007005C2640216A6F537C3E55894014003E4
:1017A8000216B00217D8C3E55B94014009855E5D57
:1017B8007562FF756301C3E55B94FA5013741F5596
:1017C8002E7004E5286009C3E53C94F05002C1B0CE
:1017D80011997887E6FE7602317E7887EEF6E4F591
:1017E80022F523F524F525F55FC2601207B2119999
:1017F800741F552E7007E528700302134A7895E682
:1018080030E009121CE5121CE5121CE5788DE6C3D0
:101818009401400302138402149C901A0D7820123C
:101828001C00E520B4A50CA3121C00E520B45A0343
:101838000218441211151218D20218D1901A0378FE
:1018480080121C00A308121C00A308121C00A30885
:10185800121C00A308A308A308121C00A308121C4A
:0F18680000A308121C00A308121C00A308A30869
:10187700A308121C00A308121C00A308121C00A333
:1018870008121C00A308121C00A308A308121C00BE
:10189700A308121C00A308121C00A308121C00A313
:1018A70008121C00A308121C00A308121C00A3089E
:1018B700121C00A308121C00A308121C00A3081284
:1018C7001C00A308121C00901A2122C2AF121C3F51
:1018D700121C19901A00740A121C05A37404121C16
:1018E70005A37410121C05901A037880121C04A318
:1018F70008121C04A308121C04A308121C04A30842
:10190700A308A308121C04A308121C04A308121C92
:1019170004A308121C04A308A308A308121C04A309
:1019270008121C04A308121C04A308121C04A30811
:10193700121C04A308A308121C04A308121C04A366
:1019470008121C04A308121C04A308121C04A308F1
:10195700121C04A308121C04A308121C04A30812D7
:101967001C04A308121C04A308121C04A308121CBD
:0B19770004121C52121C30901A212296
:101A00000A041007070104FFFF0A020101A55A0199
:101A100000B40301FF0301010225D078C8040D01C1
:021A200000FFC5
:101A4000235475726E696779323541232020202036
:101A500023424C48454C4923463333302320202031
:101A60002020202020202020202020202020202076
:101C0000E493F622E6438F01538FFD75EF0275B71B
:101C1000A575B7F1F0538FFE22438F02438F0175F4
:101C2000EF0275B7A575B7F1901A0DF0538FFC222E
:101C3000901A0D74A59105901A0E745A9105227A86
:101C40003079D07820901A409100E520F709A3DA86
:101C5000F7227A3079D0901A40E7910509A3DAF992
:101C600022AB6EA86FBB01057980021CE2BB0205A6
:101C70007981021CE2BB03057982021CE2BB0405E8
:101C80007994021CE2BB05057983021CE2BB0605C0
:101C90007995021CE2BB07057986021CE2BB0805A8
:101CA000798F021CE2BB09057990021CE2BB0A0590
:101CB0007992021CE2BB0B05799B021CE2BB0C056E
:101CC0007993021CE2BB0D057987021CE2BB0E056D
:101CD000799C021CE2BB0F057988021CE27989021B
:101CE0001CE2E8F7227C051207C6DCFB22C2AF1219
:101CF00007D51207DC1207E31207EA1207BA120728
:101D0000D51207DC1207E31207EA1207BA1207D549
:101D10001207DC1207E31207EAD2AF22C2AF1207A2
:101D2000EA1207E31207DC1207D51207BA1207EA14
:101D30001207E31207DC1207D51207BA1207EA12DC
:101D400007E31207DC1207D5D2AF22AE6EAF6FC227
:101D5000AF1207D51207D51207D51207BADEF21255
:101D600007EA1207BADFF8D2AF2291ED91E591E5CB
:101D7000756E01756F01757000B14B7C05AD581221
:101D800007C6C3ED955870F5C3E55894014009C3E3
:101D9000E55894FF4032A1A691611218D291EDC28C
:101DA000AF75EF1291E5DCD50570C3E57094035073
:101DB0000280C691E5056FE56E149000B193F808B6
:101DC000C3E56F98500280AE91E591E5056EC3E5DD
:101DD0006E94115002809C1211151218D2C2AF7568
:041DE000EF1291E588
:00000001FF
